:030000000219FDE5
:03000B000200AA46
:03002B0002016C63
:03005B000203029B
:030073000202E89E
:1000800002030406080C10182030406080040608A3
:100090000C10182030406080A0C000070F1F3F0DDB
:1000A0000D0403060D0503030202C2AFC0D0C0E079
:1000B000206217E5256002E473E525F4F58A758B67
:1000C00000D262D0E0D0D0D2AF3285268AC262E5BB
:1000D00026F4603C306803207210758B00D0E0D0AD
:1000E000D0C283C294C295D2AF32C283C294C295A9
:1000F000206E13206610740CD5E0FDE57EB5070474
:10010000429021064280758B00D0E0D0D0D2AF3231
:10011000758A00C28DD262210601B9306805206659
:1001200002D28301B9306805206602D29401B93049
:100130006805206602D29501B9C28030680A20663F
:10014000077408D5E0FDD28301B9C28230680A2065
:1001500066077408D5E0FDD29401B9C29730680AE9
:100160002066077408D5E0FDD29501B9C2AFC2ADD3
:1001700053E6EFC0D0C0E0D2D3D2AFC2CEE52A6002
:1001800007207449152A21CD7800790020742EE5C6
:1001900080307E01F430E50278FF53DACF207E0311
:1001A00043DA20307E0343DA10C2D8C271E58030D2
:1001B0007E01F430E50279FFC3E89970CB3061032A
:1001C000752A40207403752A40885FD27020740D10
:1001D000E52B6004152B21DD43DA01C2D820700223
:1001E00021F0A85F206102C27020740221EE8822F3
:1001F0007882B60403852224C3E52594404002D2C8
:100200006420CF0AD0E0D0D043E610D2AD32C2CFC6
:10021000053A7802E52A6005307402152AC3E55FC5
:1002200094014005756200413A756300756C00E504
:10023000622401F56250037562FF7982B7020D30C6
:100240006D1DC3E52294324016854D227982B70395
:100250000E306D0BC3E52294324004798E8722C3A1
:10026000E5239522600840041523416E0523D8CA72
:10027000056CE56C7002156CD56D63756D017805C4
:10028000C3E56C956E4057C3E56C956F50087801D7
:10029000756D030202A2C3E56C9570500578017577
:1002A0006D01C3E5659524401E7982B7040241D3F0
:1002B000206D14852465E56C046003856E6C756D96
:1002C0000175233C0202DEE5652850057565FF4196
:1002D000D3F565E5650470067563FF756CFFD0E0C6
:1002E000D0D043E610D2AD32C2AFC0D053E67FC209
:1002F00060759100855694855795759104D0D0D23C
:10030000AF32C2AF53E6EFC2ADC0D0C0E0C0F0D252
:10031000D3D2AFA8FBA9FCC2D8307102616953DA0D
:10032000CF207E0343DA10307E0343DA20D271E51A
:1003300080307E01F420E502614088278928A148A9
:1003400053DACF207E0343DA20307E0343DA10C233
:10035000D8C271307402A1347800E580307E01F497
:1003600030E502A134885FA11C53DACF207E03431D
:10037000DA20307E0343DA10C271206102814253D9
:10038000DACF207E0343DA10307E0343DA20C2D86E
:10039000D271885A895BC3E89558F8E99559F97B79
:1003A000007E087A00C3E8948CE994005005755EDD
:1003B000008134882178A2E6A8216055C3E894C85A
:1003C000E994005008E4D2E4FB7A0A810FC3E89470
:1003D00068E994015008E4D2E3FB7A0F810FC3E887
:1003E00094D0E994025008E4D2E2FB7A1E810FC354
:1003F000E894A0E994055008E4D2E1FB7A3C810F2F
:10040000C3E89498E994085008E4D2E0FB7A787E37
:1004100000C3E8955CFCE9955DFD30E70AECF42447
:1004200001FCEDF43400FD755E00C3EC9AED9E50C6
:1004300003755E01885C895D855A58855B59780231
:10044000A11CC3E89527F8E99528F9307C02A100A2
:10045000307B02A100307A0281F92075028165E9C2
:10046000FDE8FC8184E9C313F9E813F830790281CF
:0F047000F9E9C313F9E813F830780281F9E9C309
:10047F0013FDE813FC206126C3EC941CED9402409D
:10048F0002819BED7018C3EC94C850120529C3E587
:10049F0029940A5002A134755F00D270A134E52966
:1004AF00600215297400207F037896E624FAFEE493
:1004BF003400FFC3EC9EFCED9FFD500678007900E1
:1004CF00A100C3EC94FFED9400400678FF7900A1E2
:1004DF0000EC8575F0A4C5F0A2F733F8790040035E
:1004EF0002051C78FF790002051CE9C313F9E81314
:1004FF00F8307C0EE9600278FFC3E81338F8E43473
:10050F0000F9C3E894FFE99400400278FF885FD2B6
:10051F0070206102A134741FF4552F4BF52FC27454
:10052F00EB7002D274752A40307403752A0A306159
:10053F0002A14820740353DAFE207403752B20D0D8
:10054F00F0D0E0D0D0D2AD43E61032790102057879
:10055F007903020578790A020578791E0205787900
:10056F006402057879C80205787817E4D5E0FDD8DC
:10057F00FAD9F6227A147B7802059F7A107B8C02C7
:10058F00059F7A0D7BB402059F7A0B7BC802059FEE
:10059F007902B27DE4C282D5E0FDD294D5E0FDC2EE
:1005AF0094D5E0FDD282D5E0FDD283E576D5E0FD8E
:1005BF00C2837496D5E0FDD9D9EAF8D5E0FDD8FB12
:1005CF00DBCEC28222C37C007D0075F00005F0EA0D
:1005DF0033FAEB33FB50F6EB13FBEA13FAC3E9FFE5
:1005EF00E8FEE89AF8E99BF95004EFF9EEF8B3EC5E
:1005FF0033FCED33FDD5F0DFEDF9ECF822E889F0AF
:10060F008A20D2D4F8A9F07B0030F70B7BFFF424BB
:10061F0001F8E9F43400F9E88520F0A4ADF0F8E929
:10062F008520F0A4AFF0FEED2EF974003FFA7C04A4
:10063F00C3EA13FAE913F9E813F8DCF48BF030F797
:10064F000AE8F42401F8E9F43400F9E889F0C2D497
:10065F00F8A9F0227882B60403020702C3E55F947B
:10066F0019401EE52D54067018206D3678057994C3
:10067F00E7146007780A1460027812C3E5419840C6
:10068F001F306D09856765756CFF756D01852224B7
:10069F00E4F545F546F547F548F549C26D02070201
:1006AF00D26D7994E7147013E523F43333F913F80B
:1006BF00E9540104F9E854FE0206F6E71414701425
:1006CF00E523F4333333F913F8E9540304F9E85409
:1006DF00FC0206FEE523F433333333F913F8E95400
:1006EF00070404F9E854F8C39440F8E99400F98832
:1006FF0045894622C3E54113F9E54013F8C3E545A3
:10070F0098F8E54699F9500CC3E89480E994FF40B6
:10071F001602073AC3E8947FE99400500302073AA0
:10072F00787F790002073A788079FF884A894B22CF
:10073F00E54A2547F8E54B3548F9854B20E4300766
:10074F0001F43549FA30E709C3EA94F0401502077E
:10075F0078C3EA940F500302077878FF79FF7A0F76
:10076F00020778780079007AF0C3E5249564500A7F
:10077F00C374019524500B020796E54B20E70E0238
:10078F000796E54B30E706884789488A492278A4BF
:10079F00E6FAC3E54A33F8E54B33F9D10CE930E714
:1007AF000BC3E89480E994FF4013E1D0C3E8947F32
:1007BF00E994005002E1D0787F7900E1D078807918
:1007CF00FFE820E715C3E52398F84009C3E8940133
:1007DF0040030207F778010207F7E8F42401252305
:1007EF00F840030207F778FF884C2278A5E6FAA8AD
:1007FF0048A94912060CE930E70CC3E89401E994C3
:10080F00FF401602082CC3E894FFE994005003023E
:10081F00082C78FF790002082C780179FFE920E78E
:10082F0015C3E54C98F84009C3E89401400302084A
:10083F00537801020853E8F42401254CF8400302D1
:10084F00085378FF88242278FFC26420693D206A0C
:10085F0012D264C3E541940A4009C3E52594405080
:0E086F0002C26479A1E76023E541601F74FFB7
:10087D008541F0848539F0306A0375F005A4F8C51B
:10088D00F0600278FFC3E895675002A8678866227A
:10089D00C3E5409440E5419401E56650031401AE73
:1008AD00046002F566227883E6F520120F4D75E897
:1008BD009012055A75E890E5E820ECFBA8BDA9BE9D
:1008CD00120FE7757155757200C3740013FD7455E1
:1008DD00606613FC74552CFC74003DFDECFAEDFBC9
:1008ED00C3E89AE99B4014E5712455F571E572341E
:1008FD0000F572EA2CFAEB3DFB80E5AE71AF72C3E9
:10090D00E57213F9E57113F8C3E913F9E813F87AF1
:10091D0003C3E913F9E813F8DAF7AA201A70097579
:10092D0071007572000209451AEA6008EE28FEEFA3
:10093D0039FFDAF88E718F722275E890227883E68E
:10094D00FFE5E820ECF7A8BDA9BE0573C3E57394D8
:10095D00084052757300E9FA79A0E76044EA700720
:10096D00E574601B020980C3E895746010E574504E
:10097D0006600C1402098C0460F902098CE574F50B
:10098D0074C3946D401B7564C0C3940440137564A7
:10099D0080C39404400B756440C394044003756494
:1009AD000075BB0922EFC39401601F7455601BC312
:1009BD00E894FFE994035012C3E89571E9957250DC
:1009CD0009E564600C15640209DEE564F460020556
:1009DD0064A864C3E524985002A824C3E895654033
:1009ED000AA865E565F4600385656488258826E5B4
:1009FD0073B4070375BB1022743279A687F0A4C5B2
:100A0D00F0A2F733F8C3E895644002A86488228801
:100A1D0024882588268867227540007541F022C2FA
:100A2D00AF75C820A8CCA9CDAA3A30CF010A75C898
:100A3D0024D2AFAB3BAC3C883B893CC3E89BF8E987
:100A4D009C206908F93067026141419EAD3D8A3DA8
:100A5D00F9EA9DFA600478FF79FFAE3EAF3F8B3E19
:100A6D008C3FC3EC9FFCC3E99CF542A83BA93CC35A
:100A7D00E89EF8E99FF9C3E54113FBE54013FAE859
:100A8D002AF540E93BF54150067540FF7541FF41A0
:100A9D00E8AA40AB41AC40AD417E047F02C3EB946C
:100AAD000440021E1FC3EB940840021E1FC3ED132A
:100ABD00FDEC13FCDEF7C3EA9CFAEB9DFBEF60093E
:100ACD00C3E913F9E813F8DFF7EA28FAEB39FB8AE3
:100ADD00408B4150067BFF8B408B41C3EB94025002
:100AED0002D2673069047F0361137892E6FFC3E594
:100AFD0037948240110FC3E53794A040010FC3EF27
:100B0D00940640027F057E06E541C4540FF9E54188
:100B1D00C454F0F8E540C4540F28F8C3E89EFAE930
:100B2D009400FB4009C3EA9402EB940050047A024E
:100B3D00E4FB618DAA40AB41EBC4FEEAC4540F4EF9
:100B4D00FCC3EA9CFAEB9400FBC3E813C313F8EA69
:100B5D0028FAEB3400FB8A408B41C3EB9402400230
:100B6D00C2677806EBC4FE7B00EAC4540F4EFAC38D
:100B7D00EA98FA4005C3940250027A027892E6FF91
:100B8D00306002618D855256855357D26043E680A1
:100B9D00C3E49AF8E49BF93067028127E8FAE9FB90
:100BAD00D3E913FDE813FC88528953C3EF94036016
:100BBD0038EF20E00DE82CF8E93DF9ECFAEDFB02F9
:100BCD000BE2E828F8E939F9C3E82402F8E9340022
:100BDD00F97AFE7BFFC3EF9403400E8A548B558840
:100BED004E894F8C508D51815B885489558A4E8B1F
:100BFD004F8C508D51306920C3E53394034019E576
:100C0D0042A2E713F8E555F4240138400B20E7081C
:100C1D007554FFF42401F555815BE8FAD3E813FC14
:100C2D008852C3EF94036020EF20E007E82CF8EC26
:100C3D00FA8147E8282402F87AFEC3EF94034008AE
:100C4D008A54884E8C50815B88548A4E8C50E56B4B
:100C5D00C3335002646BF56B3060028165753402ED
:0F0C6D00D26043E680E52D54066026A840A941D9
:100C7C00C3E913F9E813F8C2AF53E67F759100C3CB
:100C8C00E498F594E499F595759104D26043E68067
:100C9C00D2AF22D265754400752000306B037520ED
:100CAC0040020CBED265754400752040306B037554
:100CBC002000D2AF7801206722E52D54066002C2D5
:100CCC0065C3E54194054013780294054008780308
:100CDC00940540027806306902780A206019E544D0
:100CEC00601530690AC3E53394034003D53406D24A
:100CFC00AFD26CA190916DD2AF0000C2AF2067262D
:100D0C00E541C3FB940F40027B0FEB2405307301CC
:100D1C0023306A02742820620123F9306902798237
:100D2C00E58BC39940B50544E59BF45440B52002CE
:100D3C00A17A30690A08C3E8940A40010881E720C7
:100D4C00650281BEC26553E67F75910030671075F0
:100D5C0094007595FE759104D26043E68081BEAE19
:100D6C0040AF41C3E49EF594E49FF595A161C3E5C2
:100D7C00339402500281BE30650281BED802A18E2E
:100D8C0081E7C26C53E67F75910085549485559527
:100D9C00759104854E56854F57D26043E680D2AF8D
:100DAC00E52D54066008206A020533020DCA306C2A
:100DBC000D206B0A2065071581158102161F2278FC
:100DCC00003064053065027801E53775F007A4F949
:100DDC00E5F028F5F0E9A2F013A2F113A2F213F555
:100DEC0037C394785003753778C3E5379538400886
:100DFC00D266C283C294C295306002C1048550563B
:100E0C00855157D26043E68022207D11C2AF7543D5
:100E1C0002C282D280D2AF759F43020FE4C2AF757B
:100E2C004302C282D297D2AF759F43020FE4307255
:100E3C0043207D20C2AF75430390014A757E04C2E6
:100E4C0095C297306204D294C158D282D2AF759FAA
:100E5C0053020FE4C2AF75430390014A757E04C27E
:100E6C0083C280306204D294C178D282D2AF759F93
:100E7C0033020FE4207D17C2AF754303900125C2E6
:100E8C0095306202D294D2AF759F53020FE4C2AF79
:100E9C00754303900125C283306202D294D2AF75A0
:100EAC009F33020FE4207D11C2AF754304C280D280
:100EBC0097D2AF759F33020FE4C2AF754304C2974C
:100ECC00D280D2AF759F53020FE4307243207D2045
:100EDC00C2AF754305900139757E01C294C2823050
:100EEC006204D283C1F4D280D2AF759F43020FE467
:100EFC00C2AF75430590015B757E80C294C282308F
:100F0C006204D295E114D297D2AF759F43020FE4DD
:100F1C00207D17C2AF75430590011BC2943062024D
:100F2C00D283D2AF759F43020FE4C2AF75430590D5
:100F3C00012FC2943062EBD295D2AF759F43020F52
:100F4C00E4207D11C2AF754306C297D282D2AF7531
:100F5C009F53020FE4C2AF754306C280D282D2AF58
:100F6C00759F33020FE4307242207D20C2AF75436F
:100F7C000190015B757E80C283C280306204D29581
:100F8C00E190D297D2AF759F33020FE4C2AF754395
:100F9C0001900139757E01C295C297306204D283EB
:100FAC00E1B0D280D2AF759F53E1E4207D16C2AF81
:100FBC0075430190012FC283306202D295D2AF7576
:100FCC009F33E1E4C2AF75430190011BC2953062BF
:100FDC0002D283D2AF759F53C26622900119757EDF
:100FEC0000C283C294C295C280C282C297C26222DE
:100FFC00788076070876070876010876040876FF6D
:10100C000876FF08760908760208760108760178DA
:10101C008C76010876000876B40876FF0876FF080F
:10102C0076FF0876030876FF0876010876FF0876C7
:10103C00250876D00876780876C80876040876FFF6
:10104C0008760108760008767A08760A0876010890
:10105C0076010876000876FF227887E6FFC272BF19
:0E106C000302D2727888C27DE630E102D27DA6
:10107A00C27E7889E630E102D27EC3EF940260082C
:10108A00758E01D273021097758E00C27322788012
:10109A00E6149000809378A4F67881E61490008094
:1010AA009378A5F67886E61490008D9378A6F6785C
:1010BA009FE6F8700108C3E8941140027811E82805
:1010CA0028F56E256E256E28F56F256E2828F57091
:1010DA00789CE67538FF75390CB402067538A07528
:1010EA00390AB4030675388275390578A3E614906F
:1010FA00009A93F569120FE722227896E6FA789712
:10110A00E6FB7888E6B40305C3EB940EFB307F0454
:10111A007A007BFFC3EB9AFCC3948250027C8275EF
:10112A0075000575EC8575F0A4C3E5F0947D40F271
:10113A0022D27F31041205697A007B007C101205E5
:10114A005FE55F2AFA74003BFBDCF37C04C3EB1314
:10115A00FBEA13FADCF7FEC27F310422E5EF20E650
:10116A00037520000520903FFFE520146006901DBE
:10117A00FF1460009304600375EF1253D9BF7581A1
:10118A00C043FF8012055A75EF0243B203E5B32448
:10119A000420E70DF521E5E320E0068521B343E3CA
:1011AA0001120FE77580F275A40D75F13F75D4DF52
:1011BA0075904F75A5B075F2F075D50075A60175D5
:1011CA00E241E4F8F6D8FD756B01120FFC121667BE
:1011DA0078988676753001C2AF12057312058312AC
:1011EA00056912058A120569120591120569121715
:1011FA008A12057312057312056EC2AF78FA79FA6C
:10120A00308507D9FBD8F7021C0011651198310304
:10121A00310478988676120FE775885075891275A9
:10122A00C82475910475D84075A82275B80275E668
:10123A0090759B80759D0075D10E75BC5875BB095C
:10124A0075BA1175E88012055AD2AF1208B353DA8B
:10125A00CF207E0343DA20307E0343DA1043DA01DB
:10126A00C2D8C271120573D2617B037A0CE55E7033
:10127A00077A0CDB030212041205692070030212BA
:10128A0004C270E55FC3940240E1E52F541F8561F3
:10129A0060F561B560D5DAD5C26153DACF207E0335
:1012AA0043DA20307E0343DA10C2D8C27178A2E64C
:1012BA007008D274E52F54E0F52FC2757529001213
:1012CA00056E307409C3E529940A4002D2751205E5
:1012DA005F78023074027800C3E55F9840F0C2AFCD
:1012EA00120583120583120583D2AF120573754D59
:1012FA000012055F788CE6C3940150030213D1E50E
:10130A0030C3940150030213D1207435C3E55F94AE
:10131A00FF50030213D1C2AF120598D2AF12056E65
:10132A00C3E55F940150EFC2AF1205831205641240
:10133A000583D2AF12056EC3E55F94FF40E9021838
:10134A000F7F05D27F310412056EC2AFC27F31040E
:10135A00AE5FC3E55F947FD2AF407612055AC2AF43
:10136A00120598D2AFDFDC313BC3EE94057897F6CD
:10137A001205731216A91217927F0AD27F3104122C
:10138A00056EC2AFC27F3104AE5FC3E55F947FD200
:10139A00AF50E612055AC2AF120583120564120550
:1013AA0083D2AFDFD6313BEE24057896F612057369
:1013BA001216A91217C112056E3104C3E55F94FF14
:1013CA005002611302180FC3E55F954D4003855F14
:1013DA004D12056E78017988E7B403027805C3E5F2
:1013EA005F98400241FBC2AF120598120598120598
:1013FA0098D2AF120573753000E4F531F532053134
:10140A00E531F470390532789AE678191460127861
:10141A003214600D787D14600878FA14600375320E
:10142A0000C3E53298401715327531B4789986763B
:10143A00C2AF120598D2AF7898867612056E120559
:10144A0064E52A7005307402410478012074027838
:10145A0006C3E55F9840A712056EE52A70030212DB
:0F146A0004C2AF120FE7E4F522F523F524F525B0
:10147900F526F56AD2AF7885E6C333F568E4F54514
:10148900F546F547F548F549F573F52CF52DF5378A
:1014990075730875BB1012055A120946E5E820EC68
:1014A900FBA8BDA9BEE97001F8887412094A7573D1
:1014B9000875BB107887E6FE760211657887EEF627
:1014C900C2AF7564FF120A058522648522658522EB
:1014D90066D2AF752201752401752501752601852E
:1014E900636C756D017888E6B40307C27D307602B6
:1014F900D27DD268D269753300120F4D120F721264
:101509000A25120A2C120A25120A2C120A2502157A
:1015190026C2AF1165D2AF75730075BB09120CB045
:10152900120663120DCB120E15120A2C120C9F30E3
:101539006D03120703206703120856306703120868
:101549009D120DCB120E3A120A2C120CB0306D03FB
:1015590012073F120DCB120EB1120A2C120C9F303A
:101569006D0312079D120DCB120ED6120A2C120C06
:10157900B0306D031207FA120DCB120F4D120A2C5F
:10158900120946120C9F120DCB120F7212094A1240
:101599000A2C30692F206B2C856764856765856304
:1015A9006C756D0179187A0CC3E533994009C269E4
:1015B900D26A8A350215CDC3E55F9401400302154D
:1015C90026021627306A1B206B18E535147004C2F1
:1015D9006AA11AF535C3E55F940140030215260295
:1015E9001627753600C3E56294014009856765854C
:1015F900636C756D01C3E56278FA98502130740403
:10160900E52A601A78F0306B058567647820C3E5B0
:1016190041985002A1260536E55F6002C12A753658
:1016290000C2AF120FE77887E6FE76021165788768
:10163900EEF6E4F522F523F524F525F526F568C23D
:1016490068D2AF12055A120FE7307406E52A700204
:101659004104788DE6C39401400241D88103901A70
:101669000D78201216EBE520B4A50CA31216EBE5B4
:1016790020B45A03021689120FFC1216A90216A8E1
:10168900901A0378807B0A1216EBA308DBF9901AEB
:101699000F788C7B181216EBA308DBF9901A272216
:1016A900C2AF12172A121704901A00740E1216F0FC
:1016B900A374041216F0A374141216F0901A037886
:1016C900807B0A1216EFA308DBF9901A0F788C7B3E
:1016D900181216EFA308DBF912173D12171B901AFF
:1016E9002722E493F622E6438F01538FFD75EF021B
:1016F90075B7A575B7F1F0538FFE22438F02438F5B
:101709000175EF0275B7A575B7F1901A0DF0538FF2
:10171900FC22901A0D74A5D1F0901A0E745AD1F0CA
:10172900227A3079D07820901A40D1EBE520F70958
:10173900A3DAF7227A3079D0901A40E7D1F009A3D9
:10174900DAF922AB77A878BB01027980BB0202796A
:1017590081BB03027982BB04027994BB05027983B8
:10176900BB06027986BB07027992BB08027987BB5F
:101779000902799CBB0A027988BB0B027989E8F7CF
:10178900227C05120573DCFB22C2AF120583120508
:101799008A12059112059812056412058312058AA9
:1017A90012059112059812056412058312058A1211
:1017B9000591120598D2AF22C2AF12059812059170
:1017C90012058A12058312056412059812059112F1
:1017D900058A1205831205641205981205911205EE
:1017E9008A120583D2AF22AE77AF78C2AF120583D2
:1017F900120583120583120564DEF212059812059B
:1018090064DFF8D2AF2212179212178A12178A755B
:1018190077017578017579001217F07C05AD5F12B3
:101829000573C3ED955F70F5C3E55F9401400AC385
:10183900E55F94FF403702185312174C1216A9128C
:101849001792C2AF75EF1212178ADCD10579C3E579
:10185900799403500280C112178A0578E5771490AC
:0D186900009F93F808C3E57898500280A80E
:1018760012178A12178A0577C3E577940C500280EF
:0F18860094120FFC1216A9C2AF75EF1212178A37
:0319FD000211666E
:101A00000E041407070104FFFF09020101A55A0192
:101A100000B4FFFFFF03FF01FF25D078C804FF01DA
:081A200000FF0A010100FFFFB5
:101A400023416C69676E424C333558232020202097
:101A500023424C48454C4923463333302320202031
:101A60002020202020202020202020202020202076
:101C0000C2AFC2D353D9BF7581C043B20343FF8073
:101C1000752438752503B1C975EF0275E24043F1AB
:101C20002053A4DF75D400D2857DFA780379E67C51
:101C300010752200752300901DD67B0675249875BB
:101C400025013085028142208508D8FBD9F9DCF7CF
:101C500081B4308508D8FBD9F9DCF781B4B189E4C7
:101C600093A3C39A6004DDC381B4DBDBB17B600264
:101C7000812B7B08E493FAA3B15CDBF87A30B15C8A
:101C8000752200752300B17BEAFCEBFDC3ED94FEE9
:101C9000400EB17B8A278B28ED30E0048A828B834B
:101CA000B17B7AC270D8C3ED94FE601350CEBD00F4
:101CB00025EC60097520007521FF0200008100A855
:101CC00027A9280809D804D90281D3B17FEA89AAB3
:101CD000F281C50D81A0C3ED94035049EDA2E092BD
:101CE000007AC5C3E5829400E583941C50902000DF
:101CF00010438F02438F0175B7A575B7F1F030001F
:101D00001FA827A9280809438F01538FFDD804D99C
:101D100002A12089AAE275B7A575B7F1F0A3A10DBC
:101D2000538FFC817C7AC1BD030CE493A3FAB140CC
:101D3000DCF8B138817C817EAA22AB23B15CEBFA5E
:101D4000EA6222752608C3E52313F523E52213F57D
:101D50002250066323A0632201D526EAB1C9B1C986
:101D600075260AEAF4200102D285300102C285B14B
:101D7000C9C3134002C201D526EB22B17FEAFB2082
:101D80008502A17F308502A184752608AE24AF2587
:101D9000C3EF13FFEE13FEB1CDB1C9C3EA13308513
:101DA000024480FA30E703632201C3E52313F523DD
:101DB000E52213F52250066323A0632201D526D91C
:101DC000E52265236523F52222AE24AF250E0FDE22
:101DD000FEDFFCD20122424C48656C693437316326
:041DE000F3300601D5
:00000001FF
